:0404000002048D3233
:01040B0032BE
:0304130002170CC1
:03041B000218EBD9
:0104230032A6
:01042B00329E
:010433003296
:01043B00328E
:010443003286
:01044B00327E
:010453003276
:01045B00326E
:03046300021DDC9B
:01046B00325E
:010473003256
:01047B00324E
:0304830002135809
:0604E6007822E4F208F2A6
:03054E000204861E
:05048600120E7480FE5F
:0E055100AA82C00212157890840075F003E4AF
:06055F0012158CD20912F6
:05056500167BD20A1212
:05056A001686C20B1211
:0A056F001691D0027B017C0F7D275E
:060579000B1CBCFF011D7C
:0E057F00EC4D70F6C0021205C2D0028A821244
:0B058D00074F78007403F275820F0224
:0205980006401B
:0C059A0075820F1205FAAA827800741F07
:0805A6005AF275820F020640B3
:0C05AE0075820F1205FAAA827800748092
:0805BA004AF275820F020640AF
:0C05C20090F23074C0F0C2F085F0237598
:0805CE0082041226057828744E
:0705D60022F20874F2F27832
:0B05DD002A7401F208E4F290F23012E0
:0205E80016B04B
:0C05EA0012169C40FBD2F085F0237582B5
:0405F60004022605D0
:0E05FA00AA8290F2307403F090F231EAF0C25F
:0B060800F085F02375820412260578AF
:06061300287422F20874B5
:0A061900F2F2782A7403F208E4F20A
:0606230090F2301216B047
:0C06290012169C40FBD2F085F023758275
:0B0635000412260590F224E0F582225A
:0E064000AA8290F2307402F090F231EAF0904B
:0A064E00F2327800E2F0C2F085F00D
:080658002375820412260578C7
:06066000287422F2087468
:0A066600F2F2782A7403F208E4F2BD
:0606700090F2301216B0FA
:0C06760012169C40FBD2F085F023758228
:040682000402260543
:0E068600AA82758260C0021205FAAB82D00211
:0C069400EA600D4303047800EBF275826D
:0406A00060020640AE
:0C06A400780074FB5BF275826002064077
:0E06B000AA82AB838A04EBC423CCC423541F5C
:0C06BE006CCC541FCC6CCC7800ECF275B6
:0E06CA008220C002C003120640D003D0027886
:0B06D80000EAC42354E0F27582210206
:0206E3000640CF
:0E06E500AA82AB838A04EBC423CCC423541F27
:0C06F3006CCC541FCC6CCC7800ECF27581
:0E06FF008200C002C003120640D003D0027871
:0B070D0000EAC42354E0F275820102F0
:02071800064099
:0E071A00AA82AB838A04EBC423CCC423541FF1
:0C0728006CCC541FCC6CCC7800ECF2754B
:0E0734008204C002C003120640D003D0027837
:0B07420000EAC42354E0F275820502B7
:02074D00064064
:07074F00AA82BA0102800535
:05075600BA02448021FD
:0C075B0078007404F275822A12064078BF
:0B0767000074B1F27582291206407880
:0A077200007405F2758228020640AB
:0C077C0078007403F275822A120640789F
:0B078800007491F2758229120640787F
:0A079300007403F27582280206408C
:0C079D0078007403F275822A120640787E
:0B07A900007491F2758229120640785E
:0A07B400007403F27582280206406B
:0C07BE00C2F085F023758204122605901D
:0807CA00F2307440F07828744D
:0707D20022F20874F2F27834
:0B07D9002A740EF208E4F290F21412F1
:0207E40016B04D
:0C07E60012169C40FBD2F085F0237582B7
:0407F20004022605D2
:0C07F600C2F085F02375820412260590E5
:08080200F2147442F07828742E
:07080A0022F20874F2F278FB
:0B0811002A740EF208E4F290F21412B8
:02081C0016B014
:0C081E0012169C40FBD2F085F02375827E
:04082A000402260599
:0C082E00C2F085F02375820412260590AC
:08083A00F2147444F0782874F4
:0708420022F20874F2F278C3
:0B0849002A740EF208E4F290F2141280
:0208540016B0DC
:0C08560012169C40FBD2F085F023758246
:040862000402260561
:0C08660090F2147490F0C2F085F023753D
:080872008204122605782874A7
:07087A0022F20874F2F2788B
:0B0881002A740EF208E4F290F2141248
:02088C0016B0A4
:0C088E0012169C40FBD2F085F02375820E
:04089A000402260529
:0C089E00AAF0AB83E5827801F208EBF2CF
:0A08AA0008EAF27806E4F27801E2B1
:0E08B400F58208E2F58308E2F5F01228F3FE63
:0E08C200A31228F3FF8E05C423CDC423541FB8
:0E08D0006DCD541FCD6DCD90F215EDF0EEC440
:0C08DE002354E0FE90F216F07801E224B2
:0E08EA0002FA08E23400FB08E2FC8A828B83EB
:0B08F8008CF01228F3FA90F219F0784F
:0C09030001E22403FB08E23400FC08E2DF
:07090F00FD7804E4F208F298
:0C091600C003C004C0058A037C00780404
:0E092200C3E29B08E264808CF063F08095F0E5
:0C093000D005D004D003503BC002780476
:09093C00E224062414F524E4343D
:04094500F2F525782A
:0C09490004E22BFF08E23CFA8D068F82CE
:0C0955008A838EF01228F3FF852482852F
:0A0961002583F07804E22401F20877
:08096B00E23400F2D00280A387
:0C0973007806E270567582301205FAE535
:0C097F008220E3101207BE7800740BF217
:08098B00758230120640803431
:0E0993007582401205FAE58220E3101207F685
:0C09A1007800740BF27582401206408052
:0109AD001930
:0E09AE007582501205FAE58220E30E12082E23
:0B09BC007800740BF2758250120640A8
:0709C70078067401F280A51F
:0109CE002206
:0C09CF00AAF0AB83E5827807F208EBF297
:0E09DB0008EAF27D0075822CC0051205FAE5CF
:0B09E90082D0055401FEBE0102800315
:0309F400020AB440
:0909F7001208667807E22402F5FB
:0A0A00002608E23400F52708E2F5AD
:060A0A002890F227E0F540
:060A100029740F5529F5C1
:050A16002A85268285FF
:060A1B0027838528F0127C
:070A2100193690F223E0F505
:030A28002B852BF0
:050A2B002C752D00AB4D
:0A0A30002CE52DC40354F8CBC403D9
:0E0A3A00CB6BCB54F8CB6BFC90F224E0C403E2
:0C0A48005407FE7F002BFBEF3CFC7807FE
:0D0A5400E2F58208E2F58308E2F5F0EB120E
:080A61001936A3EC12193678D6
:0A0A690007E22403F52E08E2340032
:080A7300F52F08E2F5307A00CE
:070A7B008526828527838593
:0A0A820028F01228F3FBEAB5030088
:0A0A8C005024EA252EFFE4352FFB6D
:0A0A9600AC3074062A2422F582E435
:0C0AA00034F2F583E0FE8F828B838CF033
:060AAC001219360A80C990
:020AB2007D01C4
:030AB4008D82220E
:0E0AB70075822C1205FAE5825401FABA010488
:040AC5007582012213
:040AC9007582002210
:040ACD0075825822B4
:0E0AD10012175790840075F003E412176BC2E1
:050ADF000C12185AC2C0
:050AE4000D121865C2AF
:040AE9000E02187071
:0C0AED0090F23E7401F090F23FE4F090B3
:0C0AF900F2407438F090F2417440F0902C
:0E0B0500F2427405F090F243E4F0C2F085F085
:080B13002375820E12260578FD
:060B1B002C7446F2087480
:0A0B2100F2F2782E7406F208E4F2F6
:060B2B0090F23E12188F4B
:0C0B310012187B40FBD2F085F023758287
:040B3D000E02260579
:0E0B410090F2467401F090F24774ACF0C2F0EE
:0A0B4F0085F02375820E122605784A
:060B59002C7446F2087442
:0A0B5F00F2F2782E7406F208E4F2B8
:060B690090F24612188F05
:0C0B6F0012187B40FBD2F085F023758249
:040B7B000E0226053B
:0D0B7F0090F2467401F090F2477401F0907E
:0B0B8C00F2487450F090F249E4F09041
:0B0B9700F24AF090F24BF0C2F085F043
:080BA2002375820E122605786E
:060BAA002C7446F20874F1
:0A0BB000F2F2782E7406F208E4F267
:060BBA0090F23E12188FBC
:0C0BC00012187B40FBD2F085F0237582F8
:040BCC000E022605EA
:0E0BD00090F23EE4F090F23F745BF0C2F085CC
:090BDE00F02375820E1226057841
:060BE7002C7446F20874B4
:0A0BED00F2F2782E7406F208E4F22A
:060BF70090F23E12188F7F
:0C0BFD0012187B40FBD2F085F0237582BB
:0A0C09000E12260590F249E0FA7879
:090C130014EAF290F248E0FA78CC
:040C1C0015EAF222C1
:0E0C200090F23EE4F090F23F7463F0C2F08573
:090C2E00F02375820E12260578F0
:060C37002C7446F2087463
:0A0C3D00F2F2782E7406F208E4F2D9
:060C470090F23E12188F2E
:0C0C4D0012187B40FBD2F085F02375826A
:0A0C59000E12260590F249E0FA7829
:090C630016EAF290F248E0FA787A
:040C6C0017EAF2226F
:0E0C700090F23EE4F090F23F7462F0C2F08524
:090C7E00F02375820E12260578A0
:060C87002C7446F2087413
:0A0C8D00F2F2782E7406F208E4F289
:060C970090F23E12188FDE
:0C0C9D0012187B40FBD2F085F02375821A
:0A0CA9000E12260590F249E0FA78D9
:090CB30018EAF290F248E0FA7828
:090CBC0019EAF290F24BE0FA781B
:090CC5001AEAF290F24AE0FA7812
:040CCE001BEAF22209
:0E0CD20090F23EE4F090F23F745FF0C2F085C5
:090CE000F02375820E122605783E
:060CE9002C7446F20874B1
:0A0CEF00F2F2782E7406F208E4F227
:060CF90090F23E12188F7C
:0C0CFF0012187B40FBD2F085F0237582B8
:0A0D0B000E12260590F249E0FA7876
:090D15000EEAF290F248E0FA78CF
:040D1E000FEAF222C4
:0E0D220090F23EE4F090F23F745DF0C2F08576
:090D3000F02375820E12260578ED
:060D39002C7446F2087460
:0A0D3F00F2F2782E7406F208E4F2D6
:060D490090F23E12188F2B
:0C0D4F0012187B40FBD2F085F023758267
:0A0D5B000E12260590F249E0FA7826
:090D650020EAF290F248E0FA786D
:040D6E0021EAF22262
:0E0D720090F23EE4F090F23F745EF0C2F08525
:090D8000F02375820E122605789D
:060D89002C7446F2087410
:0A0D8F00F2F2782E7406F208E4F286
:060D990090F23E12188FDB
:0C0D9F0012187B40FBD2F085F023758217
:0A0DAB000E12260590F249E0FA78D6
:090DB5000CEAF290F248E0FA7831
:090DBE000DEAF290F24BE0FA7824
:090DC7000AEAF290F24AE0FA781F
:040DD0000BEAF22216
:0E0DD40090F23EE4F090F23F745CF0C2F085C5
:090DE200F02375820E122605783B
:060DEB002C7446F20874AE
:0A0DF100F2F2782E7406F208E4F224
:060DFB0090F23E12188F79
:0C0E010012187B40FBD2F085F0237582B4
:0A0E0D000E12260590F249E0FA7873
:090E17001EEAF290F248E0FA78BC
:090E20001FEAF290F24BE0FA78AF
:090E29001CEAF290F24AE0FA78AA
:040E32001DEAF222A1
:0E0E360090F23E7401F090F23F74ABF0C2F007
:0A0E440085F02375820E1226057852
:060E4E002C7446F208744A
:0A0E5400F2F2782E7406F208E4F2C0
:060E5E0090F23E12188F15
:0C0E640012187B40FBD2F085F023758251
:040E70000E02260543
:060E7400E4F53DF53EF53A
:040E7A003FF540758B
:060E7E00312275320275FD
:060E8400330212194F12A7
:090E8A001E687582021205511266
:060E93000AD1120B41120E
:020E9900102720
:090E9B0012106E400B12195B12DB
:070EA4001B6443FF0280F014
:030EAB0053FFFDF5
:070EAE00121B6412195B1214
:090EB5000AB7E5827003020F394F
:0A0EBE0090003175F0401209CF12C8
:0E0EC8001072E582606B121087AE82AF8378E5
:0B0ED60022EEF208EFF2EE4F605085B4
:050EE100333C74032501
:0C0EE6003C8E828F83F08E828F83A3E508
:0A0EF20031F08E828F83A3A3E53256
:0C0EFC00FAF08E828F83A3A3A3E53CF0E4
:020F08007E0069
:040F0A00EEB53C0004
:0E0F0E0050208E077A0074042FFFE43AFA7820
:0C0F1C0022E22FF58208E23AF583EE2471
:080F280034F8E6FAF00E80DA5D
:090F30007582021210AA63FF028F
:0D0F3900121E01AE82AF83AAF0FBEEC3953D
:080F46003DFEEF953EFFEA9528
:0A0F4E003FFAEB9540FBC3EE9464FC
:0E0F5800EF9400EA9400EB94005003020EAEFA
:080F6600121E0185823D858306
:050F6E003E85F03FF597
:050F730040120CD21237
:0A0F78000D72121072E58270030280
:020F82000EAEB1
:0C0F8400121087AA82AB837822EAF208E0
:090F9000EBF2EA4B700302101BA6
:0C0F99008A828B837406F074012AF541F3
:0A0FA500E43BF542780CE2FE08E29E
:0A0FAF00FF8E04854182854283EC29
:0E0FB900F074022AFCE43BFD8F068C828D83CF
:0A0FC700EEF074032AF541E43BF557
:0A0FD10042780AE2FE08E2FF8E04F7
:0A0FDB00854182854283ECF0740426
:0E0FE5002AFCE43BFD8F068C828D83EEF074B7
:090FF300052AF541E43BF54278C2
:0A0FFC000EE2FE08E2FF8E048541BC
:0C10060082854283ECF074062AFAE43B79
:09101200FB8F068A828B83EEF04D
:0C101B007582011210AA63FF02020EAEE3
:0E29D500402020000004010203040000000066
:0E29E3000000000000000000000000000000E6
:0E29F10040202000000401020304000000004A
:0829FF000000000000000000D0
:082A07000101010101010101BF
:0704EC007508007509007599
:0604F3000A00750B007504
:0504F9000C00C200C26E
:0104FE0001FC
:0610270012290FD203C2E2
:0C102D000490DF027413F090293DE4935E
:0E103900FA74019374029374039390DF06EA35
:07104700F0D20112147BD26C
:04104E000002147513
:0510520074C8B50C009C
:0610570050047AFA800249
:02105D007A0116
:0E105F00C00212153CE582D00254032AF5822D
:01106D002260
:04106E00A200B32207
:0A107200E50BC3950A14540FF58234
:01107C002251
:0A107D00E50AC3950B540FF582221B
:0B108700121072E5827004900000223D
:0A109200E50A75F014A424A1FA7415
:09109C00F035F0FB0ABA00010B6B
:0510A5008A828B83220A
:0A10AA00AA82E50A75F014A424A13F
:0A10B400FB74F035F0FCE50A75F05E
:0A10BE0014A424A1FD74F035F0FE27
:0E10C8008D828E83A3E0FD0D8B828C83EDF074
:0A10D600E50A75F014A424A1FB74D0
:0C10E000F035F0FC8B828C83A3EA2AFA26
:0A10EC00F0740FB50A05750A0080C4
:0110F60002F7
:0210F700050AE8
:0310F90002147569
:0910FC00E509B50804900000228A
:0A110500E50875F016A4245FFAE473
:08110F0034F0FB0ABA00010BE9
:051117008A828B832297
:0A111C00E50875F016A4245FF582C3
:09112600E434F0F583E0F58222C7
:09112F007402B5080475080022E1
:0311380005082285
:0D113B0090F1E17401F090F1E274C0F090C9
:08114800F1E11214FD74012510
:051150000C4002050C3B
:011155002277
:0A115600AA82E50B75F014A424A191
:0B116000FB74F035F0FC0BBB00010C31
:0A116B00E50B75F014A424A1FD7437
:0C117500F035F0FE8D828E83A3E0541E46
:0C1181004202A204E43342028B828C8301
:0A118D00EAF0E50B75F014A424A1AC
:0B119700FA74F035F0FB8A828B8312A3
:0911A20014FD7401250C40020546
:0111AB000C37
:0111AC002220
:0711AD0030000612113BD2D5
:0211B400052212
:0711B600E50AB50B028009F8
:0911BD00758200121156D20522C0
:0A11C600E50975F016A4245FFAE4B1
:0A11D00034F0FB7826E4F28A828BEB
:0411DA008302149FD9
:0811DE00AA82BA21030211AD3F
:0A11E600BA1E25E50975F016A424D1
:0A11F0005FFBE434F0FCC003C00410
:0C11FA00121052AD82D004D0037826ED14
:08120600F28B828C8302149F1D
:05120E00BA1F0280037D
:0312130002135172
:09121600E50975F016A478242402
:08121F005FF2E434F008F21262
:0712270025D7402CE50AB5B4
:04122E000B0280151A
:0A123200121052AD827826EDF2781A
:0B123C0024E2F58208E2F58302149F13
:0A1247007826E4F27824E2F582082C
:06125100E2F58302149F88
:0C1257007824E22401FD08E23400FE8D42
:0D126300828E83E0FF74C05FFBBBC019D218
:0412700003D2029013
:0C127400F1E17401F090F1E27480F09060
:06128000F1E11214FDD2A1
:0212860005223F
:0D128800C005C00674C05FFDBD8002800679
:06129500D006D005802800
:09129B00D006D005100002800706
:0712A400750C00C204801864
:0712AB00E50AB50B028011FA
:0A12B200740FB50B05750B008002E8
:0212BC00050B20
:0512BE00750C00B204F4
:0B12C3007824E2F58208E2F583E0F5F4
:0612CE000D7401B50D00D6
:0C12D40050787B80200114C00374015F7F
:0C12E000FCA203E433FBB50404D003803F
:0112EC003FC2
:0212ED00D0032C
:0912EF007402B509047C008004BE
:0412F800E50904FC04
:0612FC00ECB50802802899
:0A130200C003EF139203C20153076A
:0C130C001EEFC313FFE50D148D828E83CD
:0C131800F07824E2F58208E2F583EFF0A3
:061324008C09D0038002D9
:02132A007B4006
:07132C00E50AB50B02800782
:071333008B8212115680119C
:0C133A0090F1E17401F090F1E2EBF09012
:05134600F1E11214FDAD
:03134B00D20522A6
:03134E000211ADDC
:06135100BA20030211ADF9
:011357002273
:04293D008000000016
:0604FF00750E00C206C2EA
:0305050007C20822
:0C135800C023C0E0C0F0C082C083C0020F
:0E136400C003C004C005C006C007C000C00121
:0E137200C0D0E4F5D0F59BE5E930E418740333
:0B138000B50E0875821E121417800BBA
:0B138B007402B50E0675821F121417C5
:0B139600E5E930E5067582201214170F
:0A13A1003006427403B50E02804FBF
:0C13AB007402B50E2390DF3BE0FABA0D8F
:0E13B7001B90DF3CE0FA20E33A90DF12E0FAF0
:0813C500530207BA070280067B
:0613CD0074F625A4502770
:0A13D30090DF3BE0FABA0D02800340
:0313DD0075E104B3
:0613E000758221121417B2
:0A13E600E5E930E705D20875E97F5C
:0A13F000E5E930E605D20775E9BF14
:0E13FA00D0D0D001D000D007D006D005D0044E
:0D140800D003D002D083D082D0F0D0E0D04D
:02141500233280
:0C141700AA8290DF3BE0FBBB1202801EAB
:0A14230090DF3BE0FBBB01028014E8
:0E142D0090DF3BE0FB600D90DF3BE0FBBB156A
:03143B0002800329
:03143E0075E10055
:0C14410075D68253D1FD750E0290DF12AB
:0C144D007407F08A821211DE75E9CFAA44
:061459000EBA020280053C
:05145F00BA0310800833
:0814640043D60275E102800687
:06146C0043D60275E10306
:03147200C206228D
:06147500D206439B032296
:0E147B0012253890DF147414F090DF137405FE
:0E148900F090DF127407F0439A017591F0D2D3
:08149700AF90F1EE7413F02296
:0C149F00AA82AB837826E2601290DF1274
:0C14AB00E4F075A2007826E2F5A475A319
:0314B700008006AC
:0614BA0090DF127407F040
:0E14C0007CD97D0074DF2DFC90F1E8ECF07C0F
:0E14CE00D990F1E9ECF08B0490F1EAECF0908B
:0D14DC00F1EBEAF090DF02E0FA0A0A0A9054
:0B14E900F1EDEAF090F1EC7480F0905F
:0914F400F1EF7410F0750E0222F4
:0E14FD00AA82AB838B0490F1E8ECF090F1E949
:0E150B00EAF07AD97B0074DF2BFA90F1EAEA5D
:0E151900F07AD990F1EBEAF090DF02E0FA0AE6
:0C15270090F1EDEAF090F1EC7420F090EF
:09153300F1EF7440F0750E032283
:0604BC00E478FFF6D8FD14
:08153C00E5B4540C600280F8D4
:0C15440085BC82743055B44407F5B42215
:0A155000AA827827E27003EA60091E
:09155A007827E2B40308BA800509
:05156300782774AAF2D4
:0B1568008ABC7827E2F5BC12153C128B
:05157300153C02153CCF
:08049A007943E94400601B7A7C
:0504A200019029D5784E
:0304A70014759336
:0A04AA00F2E493F2A308B800020583
:0804B40093D9F4DAF27593FF0D
:07050800E4F50FF510E4F526
:05050F0011F512E4F5F6
:0305140013F514C8
:0E15780053FF3F53F1FE43F32843A90453B938
:06158600FBC28BD2AF2274
:0E158C00AA82AB83ACF0FDC3EA9417EB940087
:0E159A00EC9400ED9400400D74C09A74C69B52
:0715A800742D9CE49D50012D
:0115AF002219
:0215B0007E00BB
:0E15B200C374A69A74909B74079CE49D50101D
:0E15C0000EEDC313FDEC13FCEB13FBEA13FA64
:0215CE0080E2B9
:0C15D0007839EAF208EBF208ECF208EDC2
:0E15DC00F290000BE4F5F0C002C003C004C0A2
:0B15EA0005C006121CB8858215858321
:0515F5001685F017F55A
:0C15FA0018D006D005D004D003D0027831
:0C16060039EAF208EBF208ECF208EDF211
:0E1612009021D7E4F5F0C006121CB8AC82ADF2
:0C16200083AAF0FB7857741BF20874B723
:0E162C00F208E4F208F28C828D838AF0EB1251
:0D163A00249CAA82AB83ACF0FDD006EA250B
:0816470015FAEB3516FBEC353A
:06164F0017FCED3518FD4B
:0E165500C374FF9A74019BE49CE49D50100E38
:0E166300EDC313FDEC13FCEB13FBEA13FA804E
:01167100E395
:0916720053C5E0EE42C58AC22214
:07167B0020090453C57F2282
:0416820043C58022BA
:07168600200A0453C5BF2236
:04168D0043C54022EF
:07169100300B0453C5DF22FA
:0416980043C5202204
:03169C00A2AA22DD
:0A169F00C2AAAA13AB14EA4B6002C2
:0216A900D2AAC3
:0516AB008A828B8322FE
:0C16B000AA82AB83782AE2F5F008E2453C
:0816BC00F0601F8A0F8B10780B
:0716C40028E2F51108E2F530
:0516CB0012782AE2F58F
:0A16D0001308E2F5148A828B83E010
:0416DA00F5C1D2AADA
:0116DE0022E9
:0816DF00E58290F1E3F07511C2
:0316E700E4751295
:0516EA00F1751301750C
:0A16EF00140090F1E3E0F5C1D2AA67
:0716F900E513451470FA909F
:06170000F1E4E0F5822295
:061706007582FF0216DFF0
:0E170C00C0E0C082C083C0D075D000C28B8503
:09171A001182851283E5C1F0057E
:0617230011E4B5110205FE
:0117290012AD
:08172A00151374FFB51302153D
:0117320014A2
:07173300E5134514601305E6
:06173A000FE4B50F0205EB
:011740001098
:0A174100850F82851083E0F5C1805A
:01174B00029B
:02174C00C2AA2F
:09174E00D0D0D083D082D0E0326B
:07051700E4F543F544E4F5AF
:05051E0045F546E4F57F
:0305230047F54851
:0E17570043F54043F10243F46043A90853B93F
:06176500F7C28FD2AF2293
:0E176B00AA82AB83ACF0FDC3EA9417EB9400A6
:0E177900EC9400ED9400400D74C09A74C69B71
:07178700742D9CE49D50014C
:01178E002238
:02178F007E00DA
:0E179100C374A69A74909B74079CE49D50103C
:0E179F000EEDC313FDEC13FCEB13FBEA13FA83
:0217AD0080E2D8
:0C17AF007839EAF208EBF208ECF208EDE1
:0E17BB00F290000BE4F5F0C002C003C004C0C1
:0B17C90005C006121CB885824985830C
:0517D4004A85F04BF511
:0C17D9004CD006D005D004D003D002781C
:0C17E50039EAF208EBF208ECF208EDF231
:0E17F1009021D7E4F5F0C006121CB8AC82AD12
:0C17FF0083AAF0FB7857741BF20874B743
:0E180B00F208E4F208F28C828D838AF0EB1270
:0D181900249CAA82AB83ACF0FDD006EA252A
:0818260049FAEB354AFBEC35F1
:06182E004BFCED354CFD02
:0E183400C374FF9A74019BE49CE49D50100E57
:0E184200EDC313FDEC13FCEB13FBEA13FA806D
:01185000E3B4
:0918510053FCE0EE42FC8AFA228D
:07185A00200C0453FC7F2267
:0418610043FC8022A2
:07186500200D0453FCBF221B
:04186C0043FC4022D7
:07187000300E0453FCDF22DF
:0418770043FC2022EC
:03187B00A2AB22FB
:0A187E00C2ABAA47AB48EA4B600278
:02188800D2ABE1
:05188A008A828B83221D
:0C188F00AA82AB83782EE2F5F008E24557
:08189B00F0601F8A438B4478C2
:0718A3002CE2F54508E2F517
:0518AA0046782EE2F576
:0A18AF004708E2F5488A828B83E0C7
:0418B900F5F9D2ABC0
:0118BD002208
:0818BE00E58290F1E5F07545AB
:0318C600E675467E
:0518C900F175470175F7
:0A18CE00480090F1E5E0F5F9D2AB17
:0718D800E547454870FA9056
:0618DF00F1E6E0F58222B3
:0618E5007582FF0218BE2F
:0E18EB00C0E0C082C083C0D075D000C28F851F
:0918F9004582854683E5F9F005FE
:0619020045E4B5450205B5
:011908004698
:08190900154774FFB5470215F4
:01191100488D
:07191200E54745486013059D
:0619190043E4B5430205A2
:01191F004483
:0A192000854382854483E0F5F980D9
:01192A0002BA
:02192B00C2AB4D
:09192D00D0D0D083D082D0E0328A
:0E19360020F71030F6118883A88220F507F6FE
:05194400A8837583007B
:01194900227B
:03194A00F280F731
:02194D00F02286
:0505260078317480F241
:07194F0012197012195E125B
:051956001E22021E61CB
:03195B000219F27C
:03195E0053BEFB7A
:0E196100E5BE30E6FB75C68043BE0475C700C8
:01196F002255
:0A19700075FF0075A00675F79922B7
:0C197A00121E01AA82AB83ACF0FD783194
:0A198600D3E29AF4FA7419B50200D6
:0C1990005038E5FFA2E49210400943FF2C
:07199C0010758202122935CB
:0E19A30053F7EF53FFEF758201122935A2A40E
:0A19B100920F43F71030100343FFBC
:0119BB00101B
:0C19BC00121E01AA82AB83ACF0FD783152
:0219C800EAF241
:0119CA0022FA
:0E19CB00C2AF75D69F75820A12293575FF00CE
:0E19D90075FE0075FD0075F50075F40075F3E0
:0B19E70000900064121E2D020006227A
:0E19F200E5FF20E20C75820A12293530A203AF
:031A00000219CBFD
:011A030022C0
:061A040012197AA20F2264
:031A0A00A2A32272
:041A0D0053FFFE2263
:061A1100D2A043FF0122F8
:06052B00751900C211C2A7
:06053100127832E4F278BA
:0905370033E4F2783474FFF27A27
:040540009C7B1A780E
:0605440035EAF208EBF2BB
:0C1A17007855740AF275820112243878A8
:0B1A2300567440F275820412246A78A9
:0B1A2E00557440F275820412243878D1
:051A39003474FFF222ED
:0E1A3E0090F208E0FA53027FBA215190F20CA8
:0E1A4C00E0FAA3E0FB4A6006BA0143BB00408B
:0A1A5A0090F209E0FABA2002800AB7
:051A6400BA210280140C
:051A6900BA222E801ED0
:071A6E007853744EF2087476
:081A7500F2F2900007022403C5
:071A7D007851744EF2087469
:081A8400F2F29000070223E2D8
:0C1A8C0090F20AE0FAA3E07832EAF202DD
:021A9800242404
:011A9A002229
:011A9B002228
:011A9C002227
:0C1A9D007835E2F58208E2F58312048B34
:0E1AA90090F24EE0FAA3E0FBA3E0FCA3E0FD08
:0D1AB700BA4D1DBB011ABC0017BD00142064
:051AC4001211D2121204
:0E1AC9001E01AA82AB83ACF0FD90F1E7EAF0BB
:011AD70022EC
:0A1AD80090F255E0FABA1002800403
:041AE20075820022E7
:0E1AE60090DE0E7404F090DE14E0FA30E0079B
:071AF40090DE16E0F58222EE
:041AFB0075820022CE
:0E1AFF0090DE0E7404F090DE28E0FA90DE1601
:0C1B0D00E0FB700890DE14E0FB54FEF0DA
:051B1900D2148A8222B3
:0A1B1E00AA82AB837837794BE2F31B
:0B1B2800784CEAF208EBF27582041220
:0E1B33001E6990DE16E0FA700890DE14E0FAEB
:031B410054FEF05F
:011B4400227E
:0E1B450090DE0E7404F090DE11E0FA4401F020
:081B53007440B51903D38001B1
:011B5B00C3C6
:061B5C009211751900D280
:021B620014224B
:071B6400121EE130121B12FA
:0E1B6B001E01AA82ACF0FD90F1E7E0FBEAC398
:071B79009BFA7446B502005F
:051B800050031219CB17
:0A1B850090F255E0FABA1002800158
:011B8F002233
:0B1B900090DE0E7404F0E519700B30BD
:0A1B9B00110B90DE11E0FA20E103C7
:031BA500121B45CB
:0A1BA80090DE0E7401F078337934FA
:081BB200E2F5F0E3B5F00122B9
:0E1BBA0090DE11E0FA20E03A90DE2274A1F0F5
:0E1BC8007420F0E4F0E4F090DE22F0E4F0741B
:0C1BD60002F0E4F0783390DE22E2F090A0
:0C1BE200DE22E4F090DE11E04401F07817
:0A1BEE0033E25483F27833E2FA7810
:041BF80034F2D214DD
:011BFC0022C6
:0A1BFD0090F255E0FABA10028004DD
:041C070075820022C0
:0E1C0B0090DE0E7404F090DE11E0FA30E1106D
:081C1900EA30E00475820022AC
:081C21007440C39519F58222FD
:081C29007480C39519F58222B5
:041C3100AA82AB8355
:0A1C35007838E260527440C395193C
:071C3F00FC7838E2B5040057
:061C460050047838E2FCB6
:0A1C4C00784EECF2784FEAF208EB54
:0E1C5600F2758204C002C003C004121E9ED0AC
:0C1C640004D003D002EC2AFAE43BFB7829
:091C700038E2C39CF2EC2519F5E1
:0A1C7900197440B519B6C002C0038B
:091C8300121B45D003D00280A918
:011C8C002235
:0B1C8D00E58290DE28F005197440B5D8
:051C98001903021B45C9
:011C9D002224
:061C9E007832E2F582221B
:0A1CA400AA827833E2547C4A7833B8
:021CAE00F22220
:081CB000AA827833E24AF22215
:0E2941001201000202000020FB1F0022000015
:04294F00010203017D
:0E29530009024300020100C032090400000125
:0E2961000202010005240020010424020205E8
:0E296F00240600010524010001070581030A6A
:0E297D00000109040100020A00000007050421
:0B298B0002400000070584024000002D
:01299600043C
:042997000403090428
:0E299B00260350006F006C006F006C0075008A
:0E29A900200043006F00720070006F0072008B
:0A29B7006100740069006F006E00FB
:0C29C1000C0357006900780065006C00F2
:0229CD00972948
:0229CF009B2942
:0229D100C1291A
:0229D300E60319
:072A0F008025000000000813
:0C1CB800AA82AB83ACF0FD783DEAF20894
:0C1CC400EBF208ECF208EDF2783DE2FAD9
:0B1CD000783BE2FB8AF0A4FCADF0784A
:0A1CDB0043ECF208EDF27839E2FC68
:0C1CE5008AF0A4FDAEF07841EDF208EEAC
:0A1CF100F27844E2FD7840E2FE8E36
:0A1CFB00F0ECA42D7844F27844E2E6
:071D0500F51A783FE2FE78B9
:081D0C003AE2F51B8EF0A4255C
:051D14001A7844F2788A
:071D190043E2F51C08E2F5AE
:0A1D20001D8EF0ECA4ADF0251CFEB2
:0A1D2A00ED351DFD7843EEF208EDE3
:091D3400F27843E2F51C08E2F527
:081D3D001D783EE2FF8FF0E586
:091D45001BA4AEF0251CFDEE35D7
:0A1D4E001DFE7843EDF208EEF28F5F
:0A1D5800F0EBA47840F2783EE2FBC5
:0C1D62008BF0ECA4FCADF0783EECF20835
:0A1D6E00EDF2783CE28AF0A4783C24
:0B1D7800F2783AE28AF0A4FAACF078AE
:0A1D83003AEAF208ECF27839E4F2D3
:0A1D8D00783DE4F27841E2FA08E242
:0C1D9700FB08E2FC08E2FD783DE22AFABD
:0D1DA30008E23BFB08E23CFC08E23DFD7855
:0C1DB00041EAF208EBF208ECF208EDF258
:0A1DBC007841E208E208E208E2784C
:0C1DC60039E22AFA08E23BFB08E23CFC90
:0A1DD20008E23D8A828B838CF02228
:0804C200785FE84400600A794C
:0304CA0000759327
:0604CD00F0E4F309D8FC85
:0804D30078B5E84401600C79E2
:0B04DB000290F000E4F0A3D8FCD9FA76
:0C1DDC00C0E0C000C0D075D0007845E227
:0E1DE8002401F208E23400F208E23400F208AE
:0B1DF600E23400F2D0D0D000D0E03288
:0C1E0100A2BCE433FAC2BC7845E2FB0846
:0E1E0D00E2FC08E2FD08E2FEEA24FF92BC8B34
:071E1B00828C838DF0EE22A2
:0B1E220075EDBBD2BC75EBFAD2AF220D
:041E2D00AA82AB8357
:091E31008A048B051ABAFF011B9B
:0E1E3A00EC4D60227582FAC002C003122935F9
:0E1E48007582FA1229357582FA1229357582D3
:0A1E5600F9122935D003D00280D123
:011E6000225F
:071E610075D2E875D3F122F0
:04054A00C213C21402
:011E68002257
:0E1E6900AA82E4CA25E0CA33FB74202AFA7468
:0A1E7700DE3BFB784BE2FC784CE206
:041E8100FD08E2FE78
:0E1E8500EC60131C8A828B83E0FF8D828E83BB
:081E9300F0A3AD82AE8380EAEA
:031E9B00D214223C
:0E1E9E00AA82E4CA25E0CA33FB74202AFA7433
:0A1EAC00DE3BFB784EE2FC784FE2CB
:041EB600FD08E2FE43
:0E1EBA00EC60141C8D828E83E0FFA3AD82AE1F
:091EC800838A828B83EFF080E92C
:011ED10022EE
:0C1ED200C21390DE017401F090DE0B746E
:031EDE0007F022E8
:0C1EE100121A04400E53BE7F121A0D901E
:071EED00F255E4F0C21322DC
:0E1EF40090F255E0FA7013121A1143BE8000EE
:0C1F020000000090F2557402F0121ED294
:0E1F0E0090DE06E0FA90DE02E0FBEA30E00230
:021F1C00D213DE
:0E1F1E00EA30E21690F2557404F090F256E4A8
:0C1F2C00F0C002C003121ED2D003D0028D
:061F3800EA30E102C213D1
:051F3E00EB20E0012290
:0C1F430090DE0EE4F090DE11E0FAD21403
:0E1F4F00EA30E40B90DE117480F090F256E45C
:011F5D00F093
:0D1F5E00EA30E20990DE11E4F090F256F056
:071F6B00EA20E003022094CC
:0A1F720090F256E0FBBB0102800371
:031F7C0002201A26
:0E1F7F0090DE16E0FB90F210E0FCA3E0FD8B7C
:0C1F8D00067F00C3EC9EED9F50028C0309
:071F9900784BEBF278497967
:0C1FA0004CE2F308E209F3758200C00275
:0C1FAC00C003121E69D003D0027849E285
:0E1FB8002BF208E23400F27C0090F210E0FD03
:0E1FC600A3E0FE90F210EDC39BF0EE9CA3F0A2
:0E1FD40090F210E0FBA3E0FC4B600990DE11E0
:061FE2007440F00220949F
:0E1FE80090F208E054606007C002121A9DD00B
:011FF60002E8
:0D1FF70090DE0EE4F090F256E0FB700990D1
:08200400DE117468F002209463
:0E200C0090DE117448F090F256E4F002209439
:0C201A0090DE16E0FBBB086C784B7408ED
:08202600F2784C7408F2087412
:0C202E00F2F2758200C002121E69D0029E
:0E203A0090F256E4F090F208E054607009C095
:08204800021220FFD002800704
:07205000C002121A3ED0028B
:0D20570090DE0EE4F090F256E0FB70089071
:07206400DE117460F0802919
:0E206B00BB012690F210E0FBA3E0FC4B6008E6
:0820790090DE117440F08013A9
:0D20810090DE11744AF090F256E4F08006F3
:06208E0090DE117440F029
:0D209400EA20E16690F256E0FBBB025E9090
:0E20A100F210E0FBA3E0FCC3EB9420EC9400F3
:0B20AF0050097A0A90F256E4F0800419
:0420BA007A027B200B
:0720BE00784EEBF27849793E
:0C20C5004FE2F308E209F3758200C0024C
:0E20D100C003121E9ED003D00290DE11EAF072
:0C20DF007849E22BF208E23400F27A00AB
:0E20EB0090F210E0FCA3E0FD90F210ECC39B1D
:0520F900F0ED9AA3F0D8
:0120FE0022BF
:0A20FF0090F212E4F090F213F0905A
:09210900F209E0FA740CB50200C1
:0321120050012257
:07211500EA2A2A90211C7345
:07211C000222C802237D022C
:06212300238F02237D0260
:06212900238F02221202C6
:06212F00214302238F0290
:06213500226B02223002C1
:06213B00228D02238F0239
:022141002380F9
:0E21430090F20AE0FAA3E0FBFC7D00BC01056F
:05215100BD0002801337
:08215600BC0205BD000280205F
:08215E00BC0305BD000280393D
:032166000221E172
:0721690078497441F208748B
:0C21700029F290F2107412F0A3E4F002C7
:02217C0021EC54
:04217E00EA600122F0
:0721820078497453F2087460
:0C21890029F2902955E493FCA3E493FD97
:0A21950090F210ECF0A3EDF0804D85
:0E219F008A047D00902996E493FE7F00C3EC35
:0621AD009EED9F4001229F
:0C21B300E4CA25E0CA33FBEA24CDF58223
:0C21BF00EB3429F583E493FAA3E493FBCE
:0C21CB007849EAF208EBF28A828B83E08C
:0A21D700FA90F210F0A3E4F0800B80
:0B21E100121A9B90F256E0FA700122E7
:0E21EC0090F20EE0FAA3E0FB90F210E0FCA3EC
:0E21FA00E0FDC3EA9CEB9D500890F210EAF065
:03220800A3EBF055
:07220B0090F2567402F0226C
:0E22120090F20AE0FAA3E0FB90DE00EAF0EAA8
:0622200060047A08800250
:022226007A0438
:0822280090F255EAF0022424B3
:0E22300090F20AE0FAA3E0FBBA0005BB000240
:02223E00800816
:08224000BA0124BB0021801447
:0A22480090F255E0FA7408B50200A8
:0A225200501490F2557408F0800C4F
:0B225C0090F2557410F0121A17800168
:012267002254
:0322680002242429
:0C226B0090F255E0FABA10047A018002EB
:022277007A00EB
:0822790090F212EAF0785174B2
:0A22810012F20874F2F2900001025C
:02228B0023E24C
:08228D0090F255E0FABA1000CE
:03229500500122D3
:0B22980090F20CE0FAA3E0FB7C537D09
:0C22A300298C828D83A3A3A3A3E493FCE9
:0A22AF007D00C3EA9CEB9D40012274
:0722B90078517412F2087461
:0822C000F2F29000010223E29A
:0E22C80090F208E0541FFA7B00BA0005BB003C
:0322D6000280146F
:0822D900BA0105BB0002802BD5
:0922E100BA0206BB0003022352FD
:0322EA0002237C50
:0922ED00121A0A50047A01800261
:0222F6007A006C
:0822F80090F212EAF078517433
:0A23000012F20874F2F290000202DB
:02230A0023E2CC
:08230C0090F255E0FABA10004E
:0E231400500C90F20CE0FAA3E0FB4A600122AC
:0B23220090F20CE0FAA3E0FB7C537D7E
:0C232D00298C828D83A3A3A3A3E493FC5E
:0A2339007D00C3EA9CEB9D400122E9
:0723430078517412F20874D6
:08234A00F2F29000020223E20E
:0E23520090F20AE0FAA3E0FBEA540F6002806A
:01236000017B
:012361002259
:0823620090F255E0FABA1000F8
:03236A00500122FD
:07236D0078517412F20874AC
:08237400F2F29000020223E2E4
:01237C00223E
:03237D0002242413
:0723800078517412F2087499
:08238700F2F29000021223E2C1
:01238F00222B
:03239000A2132273
:0C239300AA8CA2BD9215C2BD438C105351
:02239F008CFEB2
:0E23A100758900C2C5D2BDABBE74FC5B4401A1
:0E23AF00F5BE000000E5BE54036007D2904367
:0423BD008701C29042
:0923C100C2BDE58930E702C21338
:0C23CA00301309C002121A0AD00250CBD6
:0C23D600E5BE30E6FB8A8CA21592BD2209
:0E23E200AA82AB8390F2567402F090F210EAD9
:0C23F000F0A3EBF07851E2FA08E2FB7871
:0723FC0049EAF208EBF222AE
:0E240300AA82AB8390F2567401F090F210EAB8
:0C241100F0A3EBF07853E2FA08E2FB784D
:07241D0049EAF208EBF2228C
:0E24240090F2567401F090F210E4F0A3F02252
:0624320090F256E4F022D6
:0C243800E58290DE0EF07855E2FA7B00A1
:0E24440074072AFAE43BFBC423CAC423541FC6
:0C2452006ACA541FCA6ACA30E40244E09F
:0C245E0090DE10EAF090DE127401F02213
:0C246A00E58290DE0EF07856E2FA7B006E
:0E24760074072AFAE43BFBC423CAC423541F94
:0C2484006ACA541FCA6ACA30E40244E06D
:0C24900090DE13EAF090DE157401F022DB
:012A160000BF
:012A170000BE
:0C249C00AA82AB83ACF0FD785BEAF2088A
:0E24A800EBF208ECF208EDF27E007F007A0005
:0424B6007B007C200B
:0724BA00785EE23392167810
:0C24C1005BE225E0F208E233F208E233AF
:0E24CD00F208E233F2EE2EFEEF33FFEA33FAAE
:0924DB00EB33FB3016034306014C
:0C24E4007857C3E2F5F0EE95F008E2F541
:0E24F000F0EF95F008E2F5F0EA95F008E2F55D
:0C24FE00F0EB95F040227857D3E29EF4FA
:0E250A00B3FEB308E29FF4B3FFB308E29AF405
:0C251800B3FAB308E29BF4FB785BE244EA
:0225240001F2C2
:0C252600DC92785BE2F58208E2F58308A5
:06253200E2F5F008E222D0
:0D25380090DF2E74FEF090DF097464F090C7
:0E254500DF0A7425F090DF0BE4F090DF0F74D6
:0E25530043F090DF107487F090DF07740AF0F9
:0E25610090DF08E4F090DF0C741DF090DF0DA9
:0E256F0074DEF090DF0E7473F090DF1A74B615
:0E257D00F090DF1B7410F090DF15741DF090CD
:0E258B00DF16741CF090DF1774C7F090DF1895
:0E259900E4F090DF1974B2F090DF1C74EAF0E9
:0E25A70090DF1D740AF090DF1EE4F090DF1F3D
:0E25B5007411F090DF237488F090DF247431ED
:0E25C300F090DF257409F090DF037404F090AF
:0625D100DF047445F02256
:0625D70090DF39E0332221
:0B25DD0090DF39E0FA747F5AF582228B
:0E25E80090DF3AE0FAC2D575F002EA30E7045F
:0425F600B2D5F40462
:0625FA008430D502F40458
:0526000024B9F582225F
:02048B00E47318
:03048D0075814C2A
:0A049000122922E5826003020486AF
:07260500AA827418B502005F
:03260C0050012258
:0D260F00EA240983C0E0EA241C83C0E02215
:02261C004E5618
:02261E005E66F6
:022620006E76D4
:02262200E5E5EC
:02262400E5E5EA
:022626007E86AE
:022628008E968C
:02262A009EA66A
:02262C00AEB648
:02262E00E5E5E0
:02263000BEC624
:02263200CED602
:01263400DEC7
:02263500262657
:02263700262655
:02263900262653
:02263B00262651
:02263D0026264F
:02263F0026264D
:0226410026264B
:02264300262649
:02264500262647
:02264700262645
:02264900262643
:02264B00262641
:01264D002666
:08264E00A218928043FD012255
:08265600A218928143FD02224B
:08265E00A218928243FD042240
:08266600A218928343FD082233
:08266E00A218928443FD102222
:08267600A218928543FD202209
:08267E00A218929043FE012214
:08268600A218929143FE02220A
:08268E00A218929243FE0422FF
:08269600A218929343FE0822F2
:08269E00A218929443FE1022E1
:0826A600A218929543FE2022C8
:0826AE00A218929643FE40229F
:0826B600A218929743FE802256
:0826BE00A21892A043FF0122C3
:0826C600A21892A143FF0222B9
:0826CE00A21892A243FF0422AE
:0826D600A21892A343FF0822A1
:0726DE00A21892A443FF10B3
:0126E50022D2
:0726E600AA827418B502007E
:0326ED0050012277
:0D26F000EA240983C0E0EA241C83C0E02234
:0226FD002F3E6E
:0226FF004D5C30
:022701006B7AF1
:022703004B4B3E
:022705004B4B3C
:022707008998AF
:02270900A7B671
:02270B00C5D433
:02270D00E3F2F5
:02270F004B4B32
:022711000110B5
:022713001F2E77
:012715003D86
:02271600272773
:02271800272771
:02271A0027276F
:02271C0028286B
:02271E00282869
:02272000272769
:02272200272767
:02272400272765
:02272600272763
:0227280028285F
:02272A0028285D
:02272C0028285B
:01272E002882
:08272F00301805538FFE8003F2
:03273700438F01CC
:04273A0053FDFE222B
:08273E00301805538FFD8003E4
:03274600438F02BC
:0427490053FDFD221D
:08274D00301805538FFB8003D7
:03275500438F04AB
:0427580053FDFB2210
:08275C00301805538FF78003CC
:03276400438F0898
:0427670053FDF72205
:08276B00301805538FEF8003C5
:03277300438F1081
:0427760053FDEF22FE
:08277A00301805538FDF8003C6
:03278200438F2062
:0427850053FDDF22FF
:0827890030180553F6FE800331
:0327910043F6010B
:0427940053FEFE22D0
:0827980030180553F6FD800323
:0327A00043F602FB
:0427A30053FEFD22C2
:0827A70030180553F6FB800316
:0327AF0043F604EA
:0427B20053FEFB22B5
:0827B60030180553F6F780030B
:0327BE0043F608D7
:0427C10053FEF722AA
:0827C50030180553F6EF800304
:0327CD0043F610C0
:0427D00053FEEF22A3
:0827D40030180553F6DF800305
:0327DC0043F620A1
:0427DF0053FEDF22A4
:0827E30030180553F6BF800316
:0327EB0043F64072
:0427EE0053FEBF22B5
:0827F20030180553F67F800347
:0327FA0043F68023
:0427FD0053FE7F22E6
:0828010030180553F7FE8003B7
:0328090043F70191
:04280C0053FFFE2256
:0828100030180553F7FD8003A9
:0328180043F70281
:04281B0053FFFD2248
:08281F0030180553F7FB80039C
:0328270043F70470
:04282A0053FFFB223B
:08282E0030180553F7F7800391
:0328360043F7085D
:0428390053FFF72230
:08283D0030180553F7EF80038A
:0328450043F71046
:0328480053FFEF4C
:01284B00226A
:07284C00AA827418B5020016
:0528530050030228D033
:0D285800EA240983C0E0EA241C83C0E022CA
:02286500979A40
:022867009DA032
:02286900A3A624
:02286B00D0D0CB
:02286D00D0D0C9
:02286F00A9AC12
:02287100AFB204
:02287300B5B8F6
:02287500BBBEE8
:02287700D0D0BF
:02287900C1C4D8
:02287B00C7CACA
:01287D00CD8D
:02287E00282808
:02288000282806
:02288200282804
:02288400282802
:02288600282800
:022888002828FE
:02288A002828FC
:02288C002828FA
:02288E002828F8
:022890002828F6
:022892002828F4
:022894002828F2
:012896002819
:03289700A28022FA
:03289A00A28122F6
:03289D00A28222F2
:0328A000A28322EE
:0328A300A28422EA
:0328A600A28522E6
:0328A900A29022D8
:0328AC00A29122D4
:0328AF00A29222D0
:0328B200A29322CC
:0328B500A29422C8
:0328B800A29522C4
:0328BB00A29622C0
:0328BE00A29722BC
:0328C100A2A022B0
:0328C400A2A122AC
:0328C700A2A222A8
:0328CA00A2A322A4
:0328CD00A2A422A0
:0228D000C32221
:0728D20030180453F7DF2268
:0428D90043F720227F
:0728DD0030180453F7BF227D
:0428E40043F7402254
:0728E80030180453F77F22B2
:0428EF0043F7802209
:0E28F30020F71430F6148883A88220F507E63B
:06290100A883758300228B
:03290700E280F774
:03290A00E4932231
:02290D00E022C6
:0C290F009003E0E493FA9003E1E4937875
:07291B0027F28A8202155029
:042922007582002298
:0B29260000000000022931000000004A
:0429310000000000A2
:08293500E5826003D582EA226D
:00000001FF
